:100000000C94B2000C94DA000C94DA000C94F70B08
:100010000C94210C0C944B0C0C94DA000C94DA0028
:100020000C94DA000C94DA000C94DA000C94DA00E8
:100030000C94DA000C940E0F0C94DA000C94DA0095
:100040000C94FF0F0C94DA000C94FE110C944C12DB
:100050000C94DA000C94DA000C94DA000C94DA00B8
:100060000C94DA000C94DA0000C2010001001100C7
:1000700011000C0000E100000A002500250021000D
:10008000009600001900390039003600127A00008D
:100090001F004600460044008070000022004D0012
:1000A0004D004A00004B00003600750075007200DC
:1000B000403800004A009C009C0099008025000008
:1000C0007200EC00EC00E900C0120000E900DA0167
:1000D000DA01D70160090000D701B603B603B30304
:1000E000B0040000B3036E076E076B0758020000F0
:1000F0006E07DC0EDC0ED80E2C010000DC0EC11DDC
:10010000C11DBE1D00000000240027002A000000C1
:100110000000250028002B0000000000230026001E
:10012000290004040404040404040202020202027A
:1001300003030303030301020408102040800102AB
:10014000040810200102040810200000000700022B
:100150000100000304060000000000000000090385
:10016000B813020311241FBECFEFD8E0DEBFCDBF0E
:1001700011E0A0E0B1E0E8EAFDE202C005900D92D6
:10018000A83CB107D9F713E0A8ECB1E001C01D927B
:10019000AE3AB107E1F711E0C2E6D1E004C0229720
:1001A000FE010E948C16CE35D107C9F70E941316A6
:1001B0000C94C7160C940000CF93DF93BC018230DF
:1001C000910510F462E070E0A091AC03B091AD0332
:1001D000ED0140E050E0E0E0F0E021C0888199814D
:1001E0008617970769F48A819B81309719F093836A
:1001F000828304C09093AD038093AC03FE0134C0AE
:100200006817790738F44115510519F084179507D7
:1002100008F4AC01FE018A819B819C01E9012097D1
:10022000E9F641155105A9F1CA01861B970B049700
:1002300008F4BA01E0E0F0E02AC08D919C9111979A
:1002400084179507F9F46417750781F412968D9158
:100250009C911397309719F09383828304C09093F5
:10026000AD038093AC03FD0132964CC0CA01861BDE
:10027000970BFD01E80FF91F6193719302978D931E
:100280009C9340C0FD01828193819C01D90110970C
:10029000A1F68091AA039091AB03892B41F4809140
:1002A0008F01909190019093AB038093AA034091AA
:1002B0009101509192014115510541F44DB75EB73E
:1002C00080918D0190918E01481B590B2091AA03BA
:1002D0003091AB03CA01821B930B8617970780F0FE
:1002E000AB014E5F5F4F8417950750F0420F531FCD
:1002F0005093AB034093AA03F9016193719302C039
:10030000E0E0F0E0CF01DF91CF910895CF93DF934C
:10031000009709F450C0EC0122971B821A82A09129
:10032000AC03B091AD03109709F140E050E0AC1779
:10033000BD0708F1BB83AA83FE0121913191E20F31
:10034000F31FAE17BF0779F48D919C911197280F79
:10035000391F2E5F3F4F3983288312968D919C91D0
:1003600013979B838A834115510571F4D093AD0394
:10037000C093AC0320C012968D919C911397AD0150
:10038000009711F0DC01D3CFFA01D383C28321910E
:100390003191E20FF31FCE17DF0769F4888199814D
:1003A000280F391F2E5F3F4FFA01318320838A8146
:1003B0009B8193838283DF91CF910895A0E0B0E089
:1003C000E4EEF1E00C9492166C01009729F4CB0155
:1003D0000E94DC006C01C1C08EEF882E8FEF982E3A
:1003E0008C0C9D1C8601060F171F0815190508F4B3
:1003F000B2C0F401A081B181A617B707B8F0A5304B
:10040000B10508F4AAC0CD0104978617970708F430
:10041000A4C01297A61BB70BF801A193B193D40106
:100420006D937C93CF010E94860197C07B01EA1AED
:10043000FB0AEEEFFFEFEE0EFF1E36016A0E7B1E8B
:10044000C091AC03D091AD03AA24BB24442455240D
:100450004AC0C615D705E1F5488159814E155F059B
:10046000B8F1CA0104978E159F05B0F41296A40F37
:10047000B51FF401B183A0832A813B81411451044B
:1004800031F0D20113963C932E93129766C03093AD
:10049000AD032093AC0361C08A819B81F8019383F3
:1004A0008283425050404E195F095183408341146A
:1004B000510431F0D20113961C930E93129704C08D
:1004C0001093AD030093AC03F4017183608345C0C6
:1004D00088819981A816B90608F45C012E018A81E9
:1004E0009B819C01E901209709F0B3CF8091AA0379
:1004F0009091AB0386159705E9F4A616B706D0F4DC
:1005000020919101309192012115310541F42DB7CF
:100510003EB780918D0190918E01281B390B0217F7
:100520001307C8F41093AB030093AA03D4016D938F
:100530007C9313C0CB010E94DC00EC01009759F0C2
:10054000F40140815181B6010E94B302C6010E94AC
:1005500086016E0102C0CC24DD24C601CDB7DEB712
:10056000E0E10C94AE16FB01DC0102C001900D929B
:1005700041505040D8F70895FB01DC018D91019066
:1005800080190110D9F3990B0895FB01DC0101904A
:100590000D920020E1F708958130910529F56F5FF4
:1005A0007F4F79F58AEC91E060E071E00E94DA1506
:1005B00081ED91E065E046E020E00E94E00E8DEEE6
:1005C00091E06091930122E330E040E050E00E942E
:1005D0006E0B8CEF91E06091950122E330E040E0FA
:1005E00050E00E946E0B0895892B59F46F5F7F4F86
:1005F00041F481ED91E00E94670D8AEC91E00E9448
:100600000D16089580E090E06FEF7FEF0E94CC021E
:10061000089581E090E06FEF7FEF0E94CC02089593
:1006200080916E0290916F02009779F410929D0173
:1006300010929E0110929F0185EF92E00E943F0F61
:1006400085EF92E00E944A0F089581309105E9F408
:1006500081E080939D0180939E0180939F0180E0C3
:1006600090E0FC01E55FFD4F11821082FC01E55D29
:10067000FD4F11821082FC01E55BFD4F118210825B
:1006800002968032910569F708958230910531F420
:1006900081E080939D0110929E0118C083309105E6
:1006A00021F410929D0181E00FC08430910531F456
:1006B00010929D0110929E0181E01CC08530910531
:1006C00041F481E080939D0180939E0110929F01EF
:1006D00008958630910531F481E080939D01109258
:1006E0009E0108C08730910541F410929D0181E080
:1006F00080939E0180939F010895089739F481E0CB
:1007000080939D0180939E0180939F0108958EE0C8
:1007100061E00E94321180E161E00E94321181E1CA
:1007200061E00E9432118AE090E00E94AE100895CC
:100730008AE090E00E94AE108EE060E00E943211EC
:1007400080E161E00E94321181E161E00E9432119A
:1007500088E097E00E94AE1008958AE090E00E9441
:10076000AE1081E160E00E9432118EE061E00E94F3
:10077000321180E161E00E94321188E097E00E942E
:10078000AE1008958AE090E00E94AE1080E160E033
:100790000E9432118EE061E00E94321181E161E03D
:1007A0000E94321188E097E00E94AE1008951F93D6
:1007B000CF93DF9380919D018823D9F0CBE0D2E0E5
:1007C00010E04991599185EF92E0612F0E94DE0F70
:1007D0001F5F1031B1F70E94870385EF92E00E94FE
:1007E0004A0F8823D1F78091C2028823E1F70E9443
:1007F000C20380919E018823C9F0CBE2D2E010E0D1
:100800004991599185EF92E0612F0E94DE0F1F5FA1
:100810001031B1F70E94870385EF92E00E944A0FE2
:100820008091C2028823E1F70E94980380919F0182
:100830008823C9F0CBE4D2E010E04991599185EFCB
:1008400092E0612F0E94DE0F1F5F1031B1F70E940E
:10085000870385EF92E00E944A0F8091C2028823AD
:10086000E1F70E94AD0380919D01882321F488E087
:1008700097E00E94AE1080919E01882321F488E0C9
:1008800097E00E94AE1080919F01882321F488E0B8
:1008900097E00E94AE10DF91CF911F910895EF92E3
:1008A000FF920F931F93CF93DF938091A40161E098
:1008B0000E9432118091A40160E00E94321100E791
:1008C00012E0C0E0D0E088E2E82EF12C8091A20195
:1008D00060E00E9432118EE190E00E94AE108091A3
:1008E000A0010E94DC11F801918380838091720243
:1008F00090917302855893403CF4809170029091DE
:1009000071028558934034F0C230D10518F0F801D7
:1009100011821082F80120813181F2E02D3B3F07E6
:100920000CF404C2209709F073C0C901880F991F05
:10093000880F991F43E02538340744F190930C0247
:1009400080930B0210922C0210922B0290934C0277
:1009500080934B029093100280930F02109230020A
:1009600010922F029093500280934F0290931402A2
:100970008093130210923402109233029093540227
:1009800080935302295E334034F534C090930C02B7
:1009900080930B0210922C0210922B0210924C02A8
:1009A00010924B029093100280930F02109230022B
:1009B00010922F021092500210924F029093140244
:1009C0008093130210923402109233021092540258
:1009D000109253020FC085EF92E060E14FEF5FE0AD
:1009E0000E94DE0F85EF92E064E14FEF5FE00E942E
:1009F000DE0FA7C085EF92E060E140E050E00E948A
:100A0000DE0F85EF92E064E140E050E00E94DE0FEF
:100A1000C130D10509F095C0409172025091730226
:100A20009A01220F331F220F331FE3E045385E0780
:100A3000DCF130930E0220930D0230932E022093AE
:100A40002D0210924E0210924D0230931602209306
:100A500015024E9DC0014F9D900D5E9D900D11247D
:100A600090933602809335021092560210925502EE
:100A700030931C0220931B0230933C0220933B02D4
:100A800010925C0210925B023093260220932502A2
:100A9000309346022093450210926602109265023E
:100AA000495E534094F53EC030930E0220930D02F0
:100AB00010922E0210922D0210924E0210924D02B0
:100AC00030931602209315021092360210923502CE
:100AD000109256021092550230931C0220931B0272
:100AE00010923C0210923B0210925C0210925B0248
:100AF000309326022093250210924602109245025E
:100B000010926602109265020DC085EF92E069E1D5
:100B10004FEF5FE00E94DE0F85EF92E06EE14FEF56
:100B20005FE00CC085EF92E069E140E050E00E9498
:100B3000DE0F85EF92E06EE140E050E00E94DE0FB4
:100B4000B5C0C230D10509F06FC020917402309158
:100B50007502C901880F991F880F991F43E0253836
:100B6000340744F110921802109217029093380241
:100B700080933702909358028093570210921E027E
:100B800010921D0290933E0280933D0290935E026C
:100B900080935D02109224021092230290934402EB
:100BA000809343029093640280936302295E3340F2
:100BB00014F556C110921802109217029093380241
:100BC00080933702109258021092570210921E0220
:100BD00010921D0290933E0280933D0210925E029D
:100BE00010925D021092240210922302909344020C
:100BF0008093430231C185EF92E063E14FEF5FE004
:100C00000E94DE0F85EF92E067E14FEF5FE00E9408
:100C1000DE0F85EF92E06AE14FEF5FE00E94DE0FAA
:100C200085EF92E06DE13FC0C330D10509F03EC0D1
:100C30002091760230917702C901880F991F880FA1
:100C4000991F10921A021092190210923A021092F1
:100C5000390290935A028093590210922002109206
:100C60001F021092400210923F0290936002809304
:100C70005F021092280210922702109248021092EE
:100C800047029093680280936702295E33400CF418
:100C900027C185EF92E062E14FEF5FE00E94DE0F37
:100CA00085EF92E06CE14FEF5FE058C1C430D105B1
:100CB00009F056C12091780230917902C901880F5C
:100CC000991F880F991F909312028093110290939D
:100CD000320280933102109252021092510290938C
:100CE000220280932102909342028093410210924B
:100CF00062021092610290932A02809329029093DB
:100D00004A028093490210926A0210926902295E97
:100D100033400CF417C185EF92E066E14FEF5FE0DE
:100D20000E94DE0F85EF92E06BE1BDCF209799F531
:100D300010920C0210920B0210922C0210922B02B5
:100D400010924C0210924B021092100210920F025D
:100D50001092300210922F021092500210924F0205
:100D60001092140210921302109234021092330265
:100D7000109254021092530285EF92E060E140E03D
:100D800050E00E94DE0F85EF92E064E140E050E029
:100D90000E94DE0FB0C0C130D105D9F510920E020D
:100DA00010920D0210922E0210922D0210924E02FD
:100DB00010924D02109216021092150210923602F5
:100DC00010923502109256021092550210921C0297
:100DD00010921B0210923C0210923B0210925C0295
:100DE00010925B0210922602109225021092460287
:100DF00010924502109266021092650285EF92E011
:100E000069E140E050E00E94DE0F85EF92E06EE184
:100E1000A3C0C230D105E9F5109218021092170252
:100E20001092380210923702109258021092570214
:100E300010921E0210921D0210923E0210923D026C
:100E400010925E0210925D02109224021092230210
:100E500010924402109243021092640210926302B4
:100E600085EF92E063E140E050E00E94DE0F85EF05
:100E700092E067E140E050E00E94DE0F85EF92E0F3
:100E80006AE140E050E00E94DE0F85EF92E06DE104
:100E900063C0C330D10579F510921A02109219027D
:100EA00010923A021092390210925A02109259028C
:100EB0001092200210921F021092400210923F02E4
:100EC0001092600210925F02109228021092270284
:100ED0001092480210924702109268021092670224
:100EE00085EF92E062E140E050E00E94DE0F85EF86
:100EF00092E06CE131C0C430D10591F5109212023C
:100F0000109211021092320210923102109252028B
:100F1000109251021092220210922102109242026B
:100F200010924102109262021092610210922A0203
:100F30001092290210924A021092490210926A02FB
:100F40001092690285EF92E066E140E050E00E9475
:100F5000DE0F85EF92E06BE140E050E00E94DE0F93
:100F60008091A20161E00E94321121960E5F1F4F15
:100F7000C730D10509F0AACC0E94D70385EF92E0D3
:100F80000E944A0FDF91CF911F910F91FF90EF9038
:100F900008951F9311E00EC081ED91E00E94700D45
:100FA000682F8A3019F41093C90104C08AEC91E0CB
:100FB0000E94941581ED91E00E94910D892B61F7BB
:100FC0001F9108950E94C9078091C901882309F4DF
:100FD000A0C08AEC91E061E071E00E940E158823C8
:100FE00021F010926F0210926E028AEC91E065E09F
:100FF00071E00E940E15882331F081E090E090931B
:101000006F0280936E028AEC91E06BE071E00E94C7
:101010000E15882331F082E090E090936F02809368
:101020006E028AEC91E06FE071E00E940E15882359
:1010300031F083E090E090936F0280936E028AEC2F
:1010400091E065E171E00E940E15882331F084E0A3
:1010500090E090936F0280936E028AEC91E06AE1D7
:1010600071E00E940E15882331F085E090E09093A6
:101070006F0280936E028AEC91E061E271E00E945F
:101080000E15882331F086E090E090936F028093F4
:101090006E028AEC91E068E271E00E940E158823EE
:1010A00031F087E090E090936F0280936E028AECBB
:1010B00091E06DE271E00E940E15882331F088E026
:1010C00090E090936F0280936E028AEC91E063E36C
:1010D00071E00E940E15882341F090E080916B0230
:1010E000882309F491E090936B021092C9016091FA
:1010F0006E0270916F0281ED91E04AE050E00E9433
:10110000F8148AEC91E060E071E00E94F4150E940E
:10111000100308952F923F924F925F926F927F92A9
:101120008F929F92AF92BF92CF92DF92EF92FF92F7
:101130000F931F93DF93CF9300D000D0CDB7DEB7CE
:101140008983262E342E2A83E0906C02F0906D0263
:1011500040909701509098016090990170909A0189
:1011600080909B0190909C01AA24BB2400E010E099
:1011700043E02A81222309F46EC03981332319F414
:10118000CC24DD2427C0C8018E0D9F1D6FEF70E0B9
:101190000E944116853520F4849F9001112413C0CC
:1011A0008A3A18F020E030E00EC08555282F30E054
:1011B000C901880F991F820F931F22273327281BED
:1011C000390B21503F4F249D6001259DD00C349D4B
:1011D000D00C1124222019F41C821B8229C0C801C2
:1011E0008E0D9F1D6FEF70E00E944116853570F4E3
:1011F000282F30E0C901880F991F820F931F2227E3
:101200003327281B390B21503F4F09C08A3A18F465
:1012100020E030E004C08A5A849F90011124269D6A
:10122000C001279D900D369D900D11249C838B83CA
:10123000332009F495C0C8018E0D9F1D6FEF70E03B
:101240000E944116853508F472C08A3A10F485551B
:1012500068C08A5A70C09981992319F4CC24DD247E
:1012600027C0C8018E0D9F1D6FEF70E00E944116D0
:10127000853520F4849F9001112413C08A3A18F018
:1012800020E030E00EC08555282F30E0C901880FDE
:10129000991F820F931F22273327281B390B2150B8
:1012A0003F4F249D6001259DD00C349DD00C11240E
:1012B000222019F41C821B8229C0C8018E0D9F1D9B
:1012C0006FEF70E00E944116853520F4849F9001F5
:1012D000112413C08A3A18F020E030E00EC0855582
:1012E000282F30E0C901880F991F820F931F2227F2
:1012F0003327281B390B21503F4F269DF001279D96
:10130000F00D369DF00D1124FC83EB83332041F169
:10131000C8018E0D9F1D6FEF70E00E94411685354C
:1013200020F4849F9001112413C08A3A18F020E021
:1013300030E00EC08555282F30E0C901880F991F75
:10134000820F931F22273327281B390B21503F4F31
:10135000289DC001299D900D389D900D112402C03B
:1013600080E090E0F501E55FFD4FD182C082F5019C
:10137000E55DFD4F2B813C8131832083F501E55BE9
:10138000FD4F9183808382E090E0A80EB91E0F5E2E
:101390001F4F90E2A916B10409F0EBCEC7010196E8
:1013A00090936D0280936C028050914021F41092D2
:1013B0006D0210926C020E94D7030E94C9070F9021
:1013C0000F900F900F90CF91DF911F910F91FF9091
:1013D000EF90DF90CF90BF90AF909F908F907F90D5
:1013E0006F905F904F903F902F9008958FE00E94F4
:1013F00086112091C801222331F08130910519F422
:101400001092C80117C0892BA9F4222399F481ED09
:1014100091E069E371E00E940B1581ED91E064E4D5
:1014200071E00E940B1581ED91E00E945D0E81E05C
:101430008093C8010E94E20780916E0290916F0232
:10144000019711F40E944F0480916E0290916F02F7
:10145000029754F080919D0160919E0140919F01FF
:1014600020916B020E948A088DEE91E00E94360B5B
:101470008DEE91E00E94FF0A882301F180916E02B7
:1014800090916F02019690936F0280936E0209977C
:1014900099F490E080916B02882309F491E0909395
:1014A0006B02992319F085E090E002C081E090E0A2
:1014B00090936F0280936E020E9410038CEF91E074
:1014C0000E94360B8CEF91E00E94FF0A882311F0F6
:1014D0000C94000008950F931F9301ED11E0C801D3
:1014E00040E056E960E070E00E94750CC8016FE4CE
:1014F00071E00E940B15C8016DE571E00E940B15AB
:10150000C80161E771E00E940B15C8016FE771E047
:101510000E940B1560ED77E080E090E00E9455108E
:10152000C80164E471E00E940B1560ED77E080E093
:1015300090E00E945510C8010E945D0E81E08093EA
:10154000C8011F910F91089588E893E040E855E2A3
:1015500060E070E00E9487128091930160E00E9439
:10156000F3108091950160E00E94F3108FE060E03D
:101570000E94F31085E060E00E94F31086E061E0D5
:101580000E94F3100E946B0A8EE061E00E94F3104B
:1015900080E161E00E94F31081E161E00E94F310BC
:1015A0008EE061E00E94321180E161E00E94321120
:1015B00081E161E00E94321185EF92E060E070E02D
:1015C0000E947D0F8091A00160E00E94F310809145
:1015D000A20161E00E94F3108091A40161E00E94E9
:1015E000F31081E00E94D9118091A40160E00E9473
:1015F00032118091A20161E00E9432110895FC0134
:101600008685882319F08485811181E008951F93D0
:10161000CF93DF93EC018D850E948611182F8C8566
:101620008117E9F00E944710288139814A815B8146
:10163000621B730B840B950B2C813D814E815F8166
:10164000621773078407950750F00E94471068835C
:1016500079838A839B831C8721E030E002C020E0ED
:1016600030E0C901DF91CF911F910895CF93DF93AF
:10167000EC010E94070B892B09F588859985AA85BD
:10168000BB850097A105B10529F10E94471028816B
:1016900039814A815B81621B730B840B950B288512
:1016A00039854A855B85621773078407950790F033
:1016B0000E944710688379838A839B8318861986E2
:1016C0001A861B8681E08E8721E030E0C901DF9118
:1016D000CF9108951E8620E030E0F8CFFF920F935F
:1016E0001F938C01F62EFC01248335834683578398
:1016F00010861186128613860E944710F8016083B7
:101700007183828393838F2D0E948611F8018487D1
:10171000F5861F910F91FF9008950F931F93CF931C
:10172000DF93FC01738D76957170A685B7859585DD
:10173000772329F08C91892309F454C004C08C913B
:10174000892309F04FC08389948920E001972FEF06
:101750008F3F9207D9F7C589D689A685B7851585A4
:1017600031E060E040E050E000E0CE01202F019742
:101770002FEF8F3F9207D9F78C91812311F0632BC4
:1017800003C0832F80956823330F4F5F5F4F48302E
:10179000510559F78789908D20E001972FEF8F3FF2
:1017A0009207D9F7711160958091C0022091C10212
:1017B00090E001968F73907030E08217930779F074
:1017C000E091C002F0E0E058FD4F60838091C002DC
:1017D00090E001968F7390708093C00203C0838D58
:1017E0008160838FDF91CF911F910F9108951F9298
:1017F0000F920FB60F9211242F933F934F935F9345
:101800006F937F938F939F93AF93BF93EF93FF93C8
:1018100080917E0290917F02009711F00E948D0BC3
:10182000FF91EF91BF91AF919F918F917F916F91B8
:101830005F914F913F912F910F900FBE0F901F908E
:1018400018951F920F920FB60F9211242F933F936A
:101850004F935F936F937F938F939F93AF93BF93B8
:10186000EF93FF9380917E0290917F02009711F099
:101870000E948D0BFF91EF91BF91AF919F918F913E
:101880007F916F915F914F913F912F910F900FBE7C
:101890000F901F9018951F920F920FB60F92112460
:1018A0002F933F934F935F936F937F938F939F9368
:1018B000AF93BF93EF93FF9380917E0290917F024D
:1018C000009711F00E948D0BFF91EF91BF91AF91A6
:1018D0009F918F917F916F915F914F913F912F9148
:1018E0000F900FBE0F901F901895CF92DF92EF923E
:1018F000FF920F931F93CF93DF93EC017A018B013B
:101900001A8E198E188E1F8A1E8A1D8A1C8A1B8A9F
:1019100020E030E06901CC0CDD1CC20ED31EB60104
:10192000660F771F660F771FAB0148595F4FFA01AB
:1019300085919591A591B4918E159F05A007B1074A
:10194000E9F4FB01E459FF4F859194919C8B8B8BBB
:10195000FB01E259FF4F859194919E8B8D8BFB018A
:10196000E059FF4F85919491988F8F8BFB01EE5832
:10197000FF4F859194919A8F898F06C02F5F3F4FBB
:101980002D30310509F0C6CF8F89988D892B09F448
:1019900049C04C85463108F03DC090916800483000
:1019A00010F484E005C04E3010F082E001C081E008
:1019B000892B80936800483028F4EDE6F0E0ADE62E
:1019C000B0E00BC04E3028F0ECE6F0E0ACE6B0E062
:1019D00004C0EBE6F0E0ABE6B0E05081483040F404
:1019E00081E090E002C0880F991F4A95E2F710C08D
:1019F000242F30E04E3018F42850304002C02E50D2
:101A0000304081E090E002C0880F991F2A95E2F7EC
:101A1000852B8C93898D9A8D20E001972FEF8F3F36
:101A20009207D9F780917E0290917F028C179D07D3
:101A300081F08B8D8E7F8B8F9FB7F8941092C002B0
:101A40008091C0028093C102D0937F02C0937E0236
:101A50009FBFDF91CF911F910F91FF90EF90DF908B
:101A6000CF900895FC014485463180F5483028F434
:101A7000EDE6F0E0ADE6B0E00BC04E3028F4EBE66A
:101A8000F0E0ABE6B0E004C0ECE6F0E0ACE6B0E0DD
:101A90005081483040F481E090E002C0880F991FE7
:101AA0004A95E2F710C0242F30E04E3018F4285049
:101AB000304002C02E50304081E090E002C0880FDC
:101AC000991F2A95E2F7809585238C930895FC0150
:101AD0008BEA91E091838083CF010E94320D0895BB
:101AE00020917E0230917F022817390731F49091BE
:101AF000C1028091C002981719F42FEF3FEF0FC079
:101B0000E091C102F0E0E058FD4F20818091C102D8
:101B100090E001968F7390708093C10230E0C9010C
:101B2000089520917E0230917F022817390719F01D
:101B300020E030E00EC08091C0022091C10290E010
:101B4000805C9F4F821B910960E470E00E94411607
:101B50009C01C90108950F931F93DC0159968D9143
:101B60009C915A97892B49F481E090E013969C93BD
:101B70008E93129720E030E097C00FB7F8945B96F1
:101B80008C915B975196ED91FC91529750962C91C8
:101B9000509781FF8DC08081822B808359968D91D3
:101BA0009C915A97059620E001972FEF8F3F92075F
:101BB000D9F75B968C915B9781FF35C031E040E0AF
:101BC00050E070E010E0832F90E086239723519639
:101BD000ED91FC91529750962C915097892B29F0BA
:101BE000808120952823208303C08081822B8083DD
:101BF00059968D919C915A97212F01972FEF8F3FE6
:101C00009207D9F7330F4F5F5F4F48305105D9F630
:101C10005196ED91FC915297908150968C915097EE
:101C20008095892333C031E040E050E070E010E05F
:101C3000832F90E0862397235196ED91FC91529744
:101C400050962C915097892B21F08081822B808394
:101C500004C0808120952823208359968D919C91E2
:101C60005A97212F01972FEF8F3F9207D9F7330F04
:101C70004F5F5F4F48305105D9F65196ED91FC9179
:101C80005297808150969C915097892B80830FBFEB
:101C900059968D919C915A9720E001972FEF8F3F95
:101CA0009207D9F721E030E0C9011F910F91089503
:101CB000808120952823208371CF20917E0230914E
:101CC0007F022817390749F49FB7F8941092C00291
:101CD0008091C0028093C1029FBF089520917E022F
:101CE00030917F022817390731F49091C102809119
:101CF000C002981719F42FEF3FEF0AC0E091C1021C
:101D0000F0E0E058FD4F8081282F332727FD3095E4
:101D1000C90108951F93CF93DF93EC01162F862FEF
:101D200060E00E94F3108B8D81FD04C0812F61E083
:101D30000E9432111C87212F30E0C9018A5C9E4F1E
:101D4000FC0184918D872E5D3E4FF9016491E62F51
:101D5000F0E0EE0FFF1FE85EFE4F859194919F87A4
:101D60008E87DF91CF911F910895FF920F931F935C
:101D70008C01F62E862F61E00E94F3108F2D61E01A
:101D80000E9432118F2D90E0FC01EA5CFE4FE4913D
:101D9000D8015096EC9350978E5D9E4FFC01649154
:101DA000E62FF0E0EE0FFF1FE25FFE4F859194916A
:101DB00052969C938E9351971F910F91FF90089587
:101DC000FF920F931F938C01F62EFC011382128257
:101DD00088EE93E0A0E0B0E084839583A683B78388
:101DE0008BEA91E091838083148A138A168A158A7C
:101DF000108E178A128E118E838D2170220F8C7F88
:101E0000822B838FC801642F0E94B50EC8016F2DED
:101E10000E948A0E1F910F91FF9008951F920F92BA
:101E20000FB60F9211242F933F934F935F936F93AD
:101E30007F938F939F93AF93BF93EF93FF9380E232
:101E40008093800010926F001092C202E091C30252
:101E5000F091C402309711F078940995FF91EF91B9
:101E6000BF91AF919F918F917F916F915F914F91B2
:101E70003F912F910F900FBE0F901F901895E5EC9A
:101E8000F2E0108211821282339682E0E53FF80779
:101E9000C1F708958091C202882311F081E008956E
:101EA00080E2809380008091F602882319F01092DE
:101EB000F60202C02D9A2D98E5ECF2E080818EBDED
:101EC0000DB407FEFDCF81818EBD0DB407FEFDCFA1
:101ED000828133968EBD0DB407FEFDCF82E0E53FD3
:101EE000F80761F791E09093C20280EA8093800046
:101EF000B09A90936F0080E00895CF93DF93EC0148
:101F0000219A229A539A2A9A239A259A229A2D98AC
:101F100081E08DBD80E58CBDCB0124E09695879551
:101F20002A95E1F7262F2295207F272BE5ECF2E07A
:101F3000808321836283339692E0E53FF907C1F7FE
:101F4000CE010E944A0F80E28093800010926F00C1
:101F50001092C202299A29988093800080E1809390
:101F6000810081E090E0909389008093880082E076
:101F700090E090938B0080938A0080E090E29093B1
:101F800087008093860083E28093B00088E080938E
:101F9000B1001092B40083E08093B3008091B1004F
:101FA00081608093B1008091810081608093810085
:101FB000CE010E944A0FDF91CF9108959FE1961BB9
:101FC00083E0989FF0011124F695E795EB53FD4FC0
:101FD00090FF06C08081807F852B80834183089598
:101FE000CA0134E0969587953A95E1F7808381811F
:101FF0008F70942F9295907F892B818308951F92E3
:102000000F920FB60F9211242F933F938F939F93AC
:10201000AF93BF938091FB029091FC02A091FD02CF
:10202000B091FE023091FF020196A11DB11D232F38
:102030002D5F2D3720F02D570196A11DB11D209346
:10204000FF028093FB029093FC02A093FD02B093E9
:10205000FE028091F7029091F802A091F902B091EE
:10206000FA020196A11DB11D8093F7029093F80228
:10207000A093F902B093FA02BF91AF919F918F9113
:102080003F912F910F900FBE0F901F9018958FB713
:10209000F8942091FB023091FC024091FD02509196
:1020A000FE028FBFB901CA0108959B01AC017FB741
:1020B000F8948091F7029091F802A091F902B09102
:1020C000FA0266B5A89B05C06F3F19F00196A11DE5
:1020D000B11D7FBFBA2FA92F982F8827860F911D7A
:1020E000A11DB11D62E0880F991FAA1FBB1F6A9531
:1020F000D1F7BC012DC0FFB7F8948091F702909101
:10210000F802A091F902B091FA02E6B5A89B05C0C9
:10211000EF3F19F00196A11DB11DFFBFBA2FA92FE6
:10212000982F88278E0F911DA11DB11DE2E0880F09
:10213000991FAA1FBB1FEA95D1F7861B970B885ED4
:102140009340C8F2215030404040504068517C4F8D
:10215000211531054105510571F60895019739F0B2
:10216000880F991F880F991F02970197F1F708951B
:10217000789484B5826084BD84B5816084BD85B562
:10218000826085BD85B5816085BDEEE6F0E0808129
:1021900081608083E1E8F0E010828081826080834A
:1021A000808181608083E0E8F0E0808181608083CD
:1021B000E1EBF0E0808184608083E0EBF0E08081FF
:1021C00081608083EAE7F0E08081846080838081A1
:1021D0008260808380818160808380818068808349
:1021E0001092C1000895CF93DF93482F50E0CA01A9
:1021F0008A5C9E4FFC0134914E5D5E4FFA018491E2
:10220000882369F190E0880F991FFC01EC5FFE4F75
:10221000A591B491FC01E25FFE4FC591D491662374
:1022200051F42FB7F8948C91932F909589238C9328
:10223000888189230BC0623061F42FB7F8948C91A8
:10224000932F909589238C938881832B88832FBF2C
:1022500006C09FB7F8948C91832B8C939FBFDF911E
:10226000CF910895482F50E0CA01865B9E4FFC0134
:102270002491CA018A5C9E4FFC0194914E5D5E4F91
:10228000FA013491332309F440C0222351F1233061
:1022900071F0243028F42130A1F0223011F514C05F
:1022A0002630B1F02730C1F02430D9F404C0809139
:1022B00080008F7703C0809180008F7D80938000A5
:1022C00010C084B58F7702C084B58F7D84BD09C0EE
:1022D0008091B0008F7703C08091B0008F7D809394
:1022E000B000E32FF0E0EE0FFF1FE25FFE4FA5917D
:1022F000B4912FB7F894662321F48C91909589239B
:1023000002C08C91892B8C932FBF0895682F70E0A9
:10231000CB01865B9E4FFC012491CB018A5C9E4FD2
:10232000FC0144916E5D7E4FFB019491992319F459
:1023300020E030E03CC0222351F1233071F0243002
:1023400028F42130A1F0223011F514C02630B1F06C
:102350002730C1F02430D9F404C0809180008F77F9
:1023600003C0809180008F7D8093800010C084B571
:102370008F7702C084B58F7D84BD09C08091B00085
:102380008F7703C08091B0008F7D8093B000892F3C
:1023900090E0880F991F885E9E4FFC01A591B49133
:1023A0008C9120E030E0842311F021E030E0C9017D
:1023B00008958093A6010895982F8E3008F09E50BE
:1023C00097708091A6018295880F880F807C892B59
:1023D00080937C0080917A00806480937A00809161
:1023E0007A0086FDFCCF2091780040917900942FEF
:1023F00080E030E0282B392BC90108951F920F92FD
:102400000FB60F9211242F933F934F938F939F9367
:10241000EF93FF938091C00082FD1DC04091C600E4
:1024200020914003309141032F5F3F4F2F73307055
:1024300080914203909143032817390771F0E0918E
:102440004003F0914103E050FD4F4083309341033E
:102450002093400302C08091C600FF91EF919F91AD
:102460008F914F913F912F910F900FBE0F901F9022
:102470001895E0919403F0919503E05CFF4F8191F2
:10248000919120813181821B930B8F739070892BE6
:1024900011F00E94C90708951F920F920FB60F9274
:1024A00011242F933F938F939F93EF93FF9320914A
:1024B00084033091850380918603909187032817C8
:1024C000390731F48091C1008F7D8093C10014C021
:1024D000E0918603F0918703EC5BFC4F20818091B3
:1024E00086039091870301968F7390709093870372
:1024F000809386032093C600FF91EF919F918F9167
:102500003F912F910F900FBE0F901F901895AF9293
:10251000BF92DF92EF92FF920F931F93CF93DF93BF
:10252000EC017A018B01DD24403081EE580780E018
:10253000680780E0780711F0DD24D39491E0A92E9C
:10254000B12CEC89FD89DD2069F0C50108A002C02D
:10255000880F991F0A94E2F7808360E079E08DE3A9
:1025600090E005C0108260E874E88EE190E0A80178
:1025700097010E94541621503040404050405695DB
:1025800047953795279580E12030380720F0DD20EA
:1025900011F0DD24D6CFE889F9893083EA89FB89F7
:1025A000208319A2EE89FF89408121E030E0C90132
:1025B0000C8C02C0880F991F0A94E2F7482B4083C5
:1025C000EE89FF894081C9010D8C02C0880F991FD7
:1025D0000A94E2F7482B4083EE89FF894081C901C4
:1025E0000E8C02C0880F991F0A94E2F7482B408393
:1025F000EE89FF8980810F8C02C0220F331F0A945D
:10260000E2F7209528232083DF91CF911F910F912E
:10261000FF90EF90DF90BF90AF900895DC011C9683
:10262000ED91FC911D97E05CFF4F219131918081EC
:102630009181281B390B2F733070C9010895DC017B
:102640001C96ED91FC911D97E05CFF4F208131813C
:10265000E054F040DF01AE5BBF4F8D919C9111972C
:102660002817390719F42FEF3FEF07C08D919C9180
:10267000E80FF91F8081282F30E0C9010895DC019F
:102680001C96ED91FC911D97E05CFF4F20813181FC
:10269000E054F040DF01AE5BBF4F8D919C911197EC
:1026A0002817390719F42FEF3FEF10C08D919C9137
:1026B0001197E80FF91F20818D919C911197019638
:1026C0008F73907011969C938E9330E0C90108959A
:1026D000DC0191968C919197882339F05496ED9175
:1026E000FC915597808186FFF9CF91961C920895B1
:1026F000CF93DF93EC01EE85FF85E05CFF4F2081F7
:102700003181E054F0402F5F3F4F2F733070DF0175
:10271000AE5BBF4F8D919C91119728173907D1F36C
:10272000E05CFF4F80819181E054F040E80FF91F99
:102730006083EE85FF85E05CFF4F31832083EE8967
:10274000FF89208181E090E00F8C02C0880F991FE3
:102750000A94E2F7282B208381E089A3EC89FD8984
:1027600080818064808381E090E0DF91CF91089543
:1027700010928B0310928A0388EE93E0A0E0B0E001
:1027800080938C0390938D03A0938E03B0938F035B
:102790008BEB91E0909389038093880380E093E032
:1027A000909395038093940384E493E0909397032C
:1027B0008093960385EC90E090939903809398031F
:1027C00084EC90E090939B0380939A0380EC90E0DC
:1027D00090939D0380939C0381EC90E090939F03E2
:1027E00080939E0382EC90E09093A1038093A003DA
:1027F00086EC90E09093A3038093A20384E08093FF
:10280000A40383E08093A50387E08093A60385E07B
:102810008093A70381E08093A8030895CF92DF926D
:10282000EF92FF920F931F93CF93DF937C016B0185
:102830008A01C0E0D0E00FC0D6016D916D01D701D3
:10284000ED91FC910190F081E02DC7010995C80F31
:10285000D91F015010400115110571F7CE01DF910C
:10286000CF911F910F91FF90EF90DF90CF9008953F
:10287000CF93DF93EC016115710519F420E030E08E
:102880000FC0DB010D900020E9F71197A61BB70BD5
:10289000E881F9810280F381E02DAD0109959C0169
:1028A000C901DF91CF9108954F925F927F928F92ED
:1028B0009F92AF92BF92CF92DF92EF92FF920F93CF
:1028C0001F93DF93CF93CDB7DEB7A1970FB6F894E0
:1028D000DEBF0FBECDBF2C01742ECB01223008F419
:1028E0002AE019A231E2C32ED12CCC0EDD1E822E9D
:1028F0009924AA24BB24672D752FA50194010E9459
:10290000541679018A01C801B701A50194010E94FA
:102910002216472D461B0894C108D1084A3014F4EA
:10292000405D01C0495CF6014083E114F1040105FA
:10293000110521F07E2C5F2DC801DDCFC201B6014B
:102940000E943814A1960FB6F894DEBF0FBECDBF1B
:10295000CF91DF911F910F91FF90EF90DF90CF907B
:10296000BF90AF909F908F907F905F904F90089511
:10297000CF92DF92EF92FF920F931F93CF93DF934B
:10298000EC016A017B012115310541F4E881F981EF
:102990000190F081E02D642F09951FC02A30310588
:1029A000D1F477FF17C0E881F9810190F081E02D23
:1029B0006DE209958C0144275527BA014C195D0930
:1029C0006E097F09CE012AE00E9454149801280F55
:1029D000391F04C02AE00E9454149C01C901DF91F0
:1029E000CF911F910F91FF90EF90DF90CF900895BE
:1029F000EF92FF920F931F937B019A010027F7FC40
:102A00000095102FB801A7010E94B8141F910F91D3
:102A1000FF90EF9008950E9438140895DC01FB01A7
:102A200014968D919C911597892B31F46115710540
:102A3000A9F090E0808108C00D90BC91A02D611597
:102A4000710529F490E08C91882349F407C0CD01E9
:102A50000E94BC029C0190E0232B09F491E0892F95
:102A600008950F931F93CF93DF93EC018B016F5F5A
:102A70007F4F888199810E94DE01009711F480E0E8
:102A800005C0998388831B830A8381E0DF91CF91FE
:102A90001F910F910895CF93DF93EC018881998165
:102AA000892B29F08A819B818617970760F4CE01D4
:102AB0000E943115882341F08C819D81892B19F466
:102AC000E881F981108281E0DF91CF910895EF9242
:102AD000FF920F931F93CF93DF93EC017B016C81E7
:102AE0007D81E114F104C1F04115510599F08A018D
:102AF000060F171FB8010E944B15882369F08881C3
:102B000099812C813D81820F931FB7010E94C502DC
:102B10001D830C8381E001C080E0DF91CF911F9184
:102B20000F91FF90EF900895DF93CF9300D0CDB732
:102B3000DEB769831A82BE016F5F7F4F41E050E0CC
:102B40000E9467150F900F90CF91DF910895CF935A
:102B5000DF93EC0188819981009711F00E94860132
:102B6000198218821D821C821B821A82DF91CF91EA
:102B70000895EF92FF920F931F93CF93DF93EC0191
:102B80007B018A01BA010E944B15882321F4CE01F2
:102B90000E94A71507C01D830C8388819981B70106
:102BA0000E94C502CE01DF91CF911F910F91FF903E
:102BB000EF900895CF93DF93EC01198218821B8266
:102BC0001A821D821C821E826115710551F0DB0183
:102BD0000D900020E9F71197A61BB70BAD010E94DD
:102BE000B915DF91CF9108950F931F93182F092FD7
:102BF0006115710559F0DB010D900020E9F711977F
:102C0000A61BB70BAD010E94B91502C00E94A71503
:102C1000812F902F1F910F910895FC018081918148
:102C20000E9486010895CF93DF930E94B8100E94FE
:102C3000A40AC9E3D2E10E94F6092097E1F30E94B9
:102C40003912F9CF629FD001739FF001829FE00D8E
:102C5000F11D649FE00DF11D929FF00D839FF00D1B
:102C6000749FF00D659FF00D9927729FB00DE11DC7
:102C7000F91F639FB00DE11DF91FBD01CF011124A4
:102C8000089597FB092E07260AD077FD04D02ED091
:102C900006D000201AF4709561957F4F0895F6F7DD
:102CA000909581959F4F0895A1E21A2EAA1BBB1BF8
:102CB000FD010DC0AA1FBB1FEE1FFF1FA217B30708
:102CC000E407F50720F0A21BB30BE40BF50B661F1E
:102CD000771F881F991F1A9469F7609570958095E2
:102CE00090959B01AC01BD01CF010895AA1BBB1BB0
:102CF00051E107C0AA1FBB1FA617B70710F0A61BFC
:102D0000B70B881F991F5A95A9F780959095BC011C
:102D1000CD010895EE0FFF1F0590F491E02D099469
:102D20002F923F924F925F926F927F928F929F92DB
:102D3000AF92BF92CF92DF92EF92FF920F931F93C9
:102D4000CF93DF93CDB7DEB7CA1BDB0B0FB6F8947A
:102D5000DEBF0FBECDBF09942A88398848885F84BA
:102D60006E847D848C849B84AA84B984C884DF802B
:102D7000EE80FD800C811B81AA81B981CE0FD11D0F
:102D80000FB6F894DEBF0FBECDBFED01089511E080
:102D9000C2E6D1E004C0FE010E948C162296C43621
:082DA000D107C9F7F894FFCF39
:102DA800006F666600617564696F0072656400672C
:102DB8007265656E00626C75650079656C6C6F771D
:102DC8000076696F6C6574006379616E0077686975
:102DD8007465007368696674000D0A2B494E513D8D
:102DE800300D0A000D0A2B494E513D310D0A000DD8
:102DF8000A2B5354574D4F443D300D0A000D0A2BF2
:102E080053544E413D417564696F42616C6C0D0AC3
:102E1800000D0A2B53544F4155543D310D0A000DF6
:102E28000A2B53544155544F3D300D0A002000AE33
:102E3800030000070008000F000F000F0001010148
:102E48001200020004000100000000AB0D0E1491F6
:102E58000D700D6E0E5D0E0000000078130E140E3E
:082E6800133F131F1368130050
:00000001FF
